:1000000012C032C031C030C02FC02EC02DC02CC095
:100010002BC02AC029C028C027C026C025C0010A7D
:100020002A4B7A85FF0011241FBECFE5D2E0DEBF48
:10003000CDBF20E0A0E6B0E001C01D92AD37B20711
:10004000E1F7E1E6F0E01282ABE6B0E08EEF159664
:100050008C9315978DEF17968C93108688E5818782
:10006000612C712C65D089C0CBCF20ED37E0019792
:1000700020F0F9013197F1F7FACF089588EE93E077
:10008000F4CF81EA87B986EC86B9369A0895369A14
:100090003699FECF85B10895EF92FF920F931F938B
:1000A000CF93C82F8B018EE1E82E80E0F82ECC2371
:1000B00061F0F701849189BDC801D7DF19BCC8017F
:1000C000D4DFC801D2DFC150F2CFCF911F910F9181
:1000D000FF90EF900895CF93DF93D82F64E170E005
:1000E0008AE0DADF84EF91E0C0DF8D2F64E639D05B
:1000F000CAE06C2F36D0892F68EC70E0CDDFBEDF10
:100100008D2F6C2F2ED0D92F2CD0892F68EC70E03A
:10011000C3DFB4DF68EC70E08D2FBEDFAFDF64E1DA
:1001200070E08AE0B9DF84EF91E0DF91CF919DCF5D
:100130008FE384BBB89A81E08ABD83BF8AB58068AB
:100140008ABD97B328B3892F90E0809590958B7FD7
:10015000822B88BB96DF8CE291E087DF98DFBBDFE4
:10016000FACF991B79E004C0991F961708F0961BE7
:0E017000881F7A95C9F780950895F894FFCFFF
:00000001FF
